:100000001729A90004300428A5002A082802031D86
:100010000B28290827020430031801300319023085
:100020002505031D013012298030A100FE30B720C4
:100030000130B7207530A8003030E228A101A117A7
:10004000B000FE30B7203008B728A401AB00AC01E7
:10005000A01124080319A0151030A3000301AB0D53
:10006000AC0D0318013058202308031D2E2808006A
:10007000A401AB00AC01A01124080319A0150530A0
:10008000A3002730AA00103051200330AA00E83026
:100090005120AA0164305120AA010A3051202B08B6
:1000A0005828A9002C08A8002B08A700F62027082C
:1000B000A700A3030319A01124080319622823022F
:1000C000031869282708031DA011A0196928303ECC
:1000D000B7280800AE00051085108316051085109E
:1000E0000F30860583122E08A01894283E30A800F1
:1000F0008030E2203330AD00A8201330A8008830D3
:10010000E220A8206430E120A8206430E1202230E1
:10011000AD00A820283093200C3093200630932087
:10012000A0142E0894282014AD00201CA2288510AD
:10013000033C031CA728A7200530A800DC30E220E0
:10014000031408002014FE3C0319B5288514201C54
:10015000201005140F3086052D08F039860405108F
:10016000AD0E2018A8283230E1202E081229A11B3C
:100170006A2883169B0083161C141A089B0A1229EE
:1001800083169A001C1555309D00AA309D009C14C2
:100190009C18C8281C119B0A122983178001840A05
:1001A000FF3E031DCE281229AA01A900FF30A9078E
:1001B000031CAA07031C12290330A800E530E22023
:1001C000D628A801F63EA700A809031CED28FE309A
:1001D0000000A7070318E828A7070000A80FE728D2
:1001E00000002718F3282718F5280800AC01AB01F8
:1001F0001030AD00280DAB0DAC0D2908AB022A085C
:10020000031C2A0FAC0203180C292908AB072A0883
:1002100003182A0FAC070310A70DA80DAD0BFA2881
:100220002708122983138312031300000800A0017A
:1002300007309F00E33083168500FB308600811372
:10024000831285018601203084006030CE20A030EA
:1002500084005030CE20203084003030CD20051571
:10026000851505160130AA00F430D520142054302D
:100270006A2072306A2061306A206E306A207330E2
:100280006A2063306A2076306A2065306A207230D6
:100290006A2020306A204E306A204C306A2020309C
:1002A0006A2056306A202D306A2032306A20803031
:1002B000A100C0301E2077306A206A206A202E30CC
:1002C0006A2070306A2069306A2063306A206230A8
:1002D0006A2061306A2073306A2069306A20633096
:1002E0006A202E306A206E306A206C306A20073017
:1002F000AA00D030D520142049306A204E306A2020
:1003000053306A2054306A2045306A204C306A20CD
:100310003D306A204B306A2065306A2075306A2093
:100320007A306A2065306A208030A100C0301E20FB
:100330005A306A2045306A204E306A2044306A20A4
:100340003D306A2056306A2065306A2072306A205B
:1003500064306A2065306A2072306A2020306A205A
:1003600067306A2061306A206A206E306A2003019B
:10037000B920A6002608013A01390319B312031D5A
:10038000B316861C0A2A0A30D4200301B31A01309E
:10039000013A0319B312031DB3168D301E20A101BB
:1003A000B31ED92952306A2043306A2035306A2082
:1003B000DF2952306A2043306A2036306A2006181E
:1003C000E329B422DF29030106180130B20003013A
:1003D0008618013032050319EF29B422E329803051
:1003E000A100C5301E2042306A2065306A20763078
:1003F0006A2065306A2073306A2074306A20693060
:100400006A2067306A2065306A206E306A202030AA
:100410006A20C12986180D2A0A2A0301B920A600DC
:100420002608B31A013C03191C2A83169B010301F9
:100430008312B31A0130C020B31E262A7F30BE00BB
:100440001F30BF000130B920C4002D2AFF30BE008C
:10045000FF30BF000230B920C4000130BA003A08B2
:10046000B700B31514206E22D92AB601B501341590
:10047000861D341103018619013E3419013C03190C
:100480000130031D0301B2003608A8003508A7009B
:100490000130AA001330012032050319532AB50A8E
:1004A0000319B60A3A2A3608013A133003193506F9
:1004B000031D5B2AD82CB31C692A8310341D8314B6
:1004C00083183415831C34110230A8007130E220E7
:1004D0006D2A0430A8004C30E22008008030A100D2
:1004E00080301E2053306A2079306A2073306A20B1
:1004F0003A306A204108382020306A206A20803053
:10050000A100C0301E2043306A206F306A206D3059
:100510006A203A306A203708382020306A206A2062
:10052000B31EA32A8030A10089301E200530A4000C
:10053000410826208030A100C8301E200630A400CB
:1005400037082620B32A8030A10088301E200830CA
:10055000A400410826208030A100C8301E200830A9
:10056000A4003708262008000A30D420BD0A333002
:100570003D02031CC42ABD01030105190130013AE3
:1005800003190511031D05150800013006180301A4
:10059000B20001304502030103180130320503198E
:1005A000D82AC5030230D4208618D72AD82AC52ACB
:1005B00008003315B31C3311051585150301861882
:1005C0000130B20003010618013032050319EB2A8D
:1005D000FA30C0003313030186180130B200030162
:1005E000061801303205B2000301861901303205C8
:1005F0000319FB2AEB2A8619FF2AA42B0C2B0A309D
:10060000D420030186180130B2000301061801301E
:10061000320503190C2BD92A0618742B8618112BB6
:10062000E32CB410FA304002031D352BC830C6004D
:10063000013006180301B20001304602030103181D
:10064000013032050319282B0530D420C603182B9E
:10065000013046020318352B0301B3190130013A6A
:100660000319B311031DB3153317B31D4A2B851A94
:10067000422B33163F0844020318402BC40A412B77
:10068000C401492B3E083A020318482BBA0A492BE9
:10069000BA015C2B851A552B3316C4080319522B4B
:1006A000C403542B3F08C4005C2BBA0803195A2B0F
:1006B000BA035C2B3E08BA003A08B7004408C100F0
:1006C0006E22331F732B4008C500C522FA3040024A
:1006D000031D6D2BFA30C500C5220B304002031CF0
:1006E000732B0A30C002A32B8618A32B331E882B32
:1006F0003312B31E822B013083169B0083124408F1
:10070000C020882B023083169B0083124408C0202F
:10071000030134180130013A03193410031D341455
:1007200034180516341C05128618A32B0511B31AAC
:100730009B2B57259C2B002505150618A02BE32C79
:100740005230D420942BD92AB601B5010130861934
:100750000301B2003608A8003508A700FF30AA0040
:10076000DC30012032050319B92BB50A0319B60A8A
:10077000A62B3310B3103608031DC42B1E303502D0
:100780000318C42BD92AFC2B3608031DCB2B2D3084
:100790003502031CD72B3608031DD72B3D303502FD
:1007A0000318D72B0830A8004D30E220FC2B360868
:1007B000031DDE2B5A303502031CEB2B3608031DBC
:1007C000EB2B6F3035020318EB2B33140530A800E8
:1007D0000301E220FC2B3608031DF22B8230350288
:1007E000031CFB2B3608031DFB2BB5303502031809
:1007F000FB2BB314FC2BD92A3808B9004208C300DC
:10080000B801C2010511B31C352C861D082C052C1E
:1008100086190B2C082C861D0E2C0B2C8619112CDE
:100820000E2C861D142C112C0730A800D030E2208D
:1008300086190516861D05120301051A013E861943
:10084000013C031D242C1C2C0430A8004C30E22059
:100850003522C217341DC21335224217341D4213EC
:100860003522C216341DC2123A2C3522341905160F
:10087000341D051235224216341D42123522C2158E
:10088000341DC21135224215341D42113522C214C5
:10089000341DC21035224214341D4210B31C582C92
:1008A0003522B817341DB81335223817341D3813C4
:1008B0003522B816341DB81235223816341D3812B8
:1008C0003522B815341DB81135223815341D3811AC
:1008D0003522B814341DB81035223814341D3810A0
:1008E000331C732C381742084302031D0130B20039
:1008F00038083902031D01303204B2000301B31875
:10090000013E3319013C031D01303204B2000130B5
:10091000B418030132040319D72C1420331C992C6A
:1009200052306A2043306A2035306A2058306A20BD
:10093000A82CB31CA22C52306A2043306A203630D7
:100940006A20A82C52306A2043306A2035306A2051
:1009500020306A2050306A2072306A206F306A205E
:1009600074306A206F306A2063306A206F306A20EA
:100970006C306A200330AA00E830D520B31CC22CAA
:10098000B312C32CB3163808B7004208C1001420B4
:100990006E22B4144208C4003808BA003414B31FDD
:1009A0003410B315B31CD62CB312D72CB316D92AD6
:1009B000051585110330AA00E830D5203908B800A4
:1009C0004308C200D92A142048306A2065306A20C2
:1009D00072306A2073306A2074306A2061306A2075
:1009E00072306A2074306A20013006180301B200A8
:1009F00001308618030132040319FF2CF42C20293E
:100A000039253A1F39253A1B362534183925341C27
:100A10003625441A3925441E3625C4193925C41DE6
:100A2000362544193925441D3625C4183925C41CDA
:100A3000362544183925441C3625BA1A3925BA1EDC
:100A400036253A1A39253A1E3625BA193925BA1DDE
:100A500036253A1939253A1D3625BA183925BA1CD2
:100A600036253A1839253A1C3625080047253C25F5
:100A700008003C2547250800FF30BC0000000000AE
:100A80000000000000000000BC0B3E2D08002030DC
:100A9000BB0000000F30BC00BC0B4C2D0615053010
:100AA000BC00BC0B512D0611BB0B492D0800BB250A
:100AB000BB25BB25BB25BB25BB25B425B425B1254E
:100AC000AE25AE25AE25341CBB25341CBB25B42574
:100AD000B4253418BB253418BB25C41BB125C41F4D
:100AE000AE25441BB125441FAE25C41AB125C41E32
:100AF000AE25441AB125441EAE25C419B125C41D26
:100B0000AE254419B125441DAE25C418B125C41C19
:100B1000AE254418B125441CAE25BA1BB125BA1F19
:100B2000AE253A1BB1253A1FAE25BA1AB125BA1E19
:100B3000AE253A1AB1253A1EAE25BA19B125BA1D0D
:100B4000AE253A19B1253A1DAE25BA18B125BA1C01
:100B5000AE253A18B1253A1CAE250800B425BB25B0
:100B60000800BB25B4250800E130BC0000000000EF
:100B7000BC0BB62D08001030BB0000000F30BC00CD
:100B8000BC0BC02D06150530BC00BC0BC52D0611D5
:060B9000BB0BBD2D0800A7
:02400E00023F6F
:06420000000000000000B8
:00000001FF
